:020000040000FA
:0400000087EF00F096
:0800080096D00B6E960E036EFC
:10001000980E046E55D8D8B4CA90D8A4CA80FC0FE4
:10002000D8A0CA92D8B0CA82800E036E960E046E13
:10003000980E076E086ACAB025D8CAB223D842D82B
:100040000304CB6E03C005F004C006F00050096E37
:100050000A6E003C0A6A4BD808500B2E0AD0BE6EBE
:100060000C0EBD6E07BEBD8A07BCBD889394CA84C2
:100070001200BB6E0C0EBA6E07BEBA8A07BCBA88F5
:100080009492F5D700D8D890073204320332120088
:10009000066A056EFF0E0526062200D0D8A01200C3
:1000A000030E046EE70E02D8F5D7046AFE0F036E46
:1000B000E86A045AD8A012000000030600D0F8D75E
:1000C000086A076A100EF36E0434073608360550C6
:1000D000075C0650085805E30550075E0650085AAD
:1000E000D88003360436F32EEFD7035012000550A4
:1000F0000902F3CF07F0F4CF08F006500902F350DD
:10010000082605500A02F350082607501200F86A24
:100110004F0EAF6E240EAC6E900EAB6E0001C69A01
:10012000400E926EE00E936EC00E946E070EB46E8B
:100130000F0EC16E59D09EAA1BD0060EAB1412E151
:10014000E1CF26F0E2CF27F0282A1EEE80F02850DB
:10015000E126000EE222AECFE7FF26C0E1FF27C076
:10016000E2FF1100AE50AE50AB98AB8811000AD040
:10017000F2A408D0F294104A112A82700F6AD6CFE6
:100180000EF0110011002850295C14E0292AE9CF53
:1001900003F0EACF04F00EEE80F02950E926000EBD
:1001A000EA22EF50036E03C0E9FF04C0EAFFD880E3
:1001B000120004D0E868036ED8A012001200286A6A
:1001C000296A9D8AF28EF28C12009D9A0EEE80F0C2
:1001D000000EEE6AE82EFDD7286A296A9D8A120071
:1001E0009EA8FED7AD6E1200929489949292899245
:1001F000929089909296899692988998929A899AE3
:1002000094908B9093968A9693948A9493928A92E0
:1002100093908A90949A8B9A94988B9893988A98B2
:10022000006A280E056E260E066E020EEEDE006ACD
:10023000280E056E260E066E010EE7DE94908B806A
:10024000320E26DF94908B90216A226AB8DFBDDFE0
:10025000CD6AF294F28A870ED56E95DF126E9D0EEE
:10026000125C09E3FE0E125C03E330EF04F003D0EE
:10027000146A30EF04F012AE12D0146A8C0E125CC5
:1002800005E112C014F01568166807D09C0E125CC8
:1002900004E112C014F01768186830EF04F014522B
:1002A00004E130EF04F030EF04F08C0E145CD8A4BD
:1002B00053D0152803E112C015F04AD012C016F031
:1002C0003C0E155C03E12190899441D03D0E155CF4
:1002D00003E1219289923BD03E0E155C03E121940B
:1002E000899035D03F0E155C03E1219689962FD079
:1002F000400E155C03E12198899829D0410E155CC8
:1003000003E1219A899A23D0480E155C03E12290DB
:100310008A961DD0490E155C03E122928A9417D06B
:100320004A0E155C03E122948A9211D04B0E155CA3
:1003300003E122968A900BD04C0E155C03E12298C3
:100340008B9A05D04D0E155C02E1229A8B981568A8
:1003500030EF04F030EF04F09C0E145CD8A430EFC2
:1003600004F0172804E112C017F030EF04F012C0B7
:1003700018F01852D8A44CD03C0E175C03E1219021
:10038000899441D03D0E175C03E1219289923BD0C4
:100390003E0E175C03E12194899035D03F0E175C27
:1003A00003E1219689962FD0400E175C03E1219836
:1003B000899829D0410E175C03E1219A899A23D0AC
:1003C000480E175C03E122908A961DD0490E175CF7
:1003D00003E122928A9417D04A0E175C03E122941B
:1003E0008A9211D04B0E175C03E122968A900BD0B3
:1003F0004C0E175C03E122988B9A05D04D0E175CCA
:1004000002E1229A8B98176830EF04F02FEF04F086
:100410003C0E175C2EE12180D6CF0EF0D7CF0FF027
:100420003C0E18240C6E0D6A0D3618500C24016E0B
:10043000000E0D20026E01C02AF002C02BF02AC06F
:1004400001F02BC002F001500E24196E02500F2053
:100450001A6E000E10201B6E000E11201C6E1BC0A9
:1004600042F01CC043F019C05AF01AC05BF08984F6
:10047000F6D13D0E175C2EE12182D6CF0EF0D7CFFC
:100480000FF03C0E18240C6E0D6A0D3618500C241B
:10049000016E000E0D20026E01C02CF002C02DF086
:1004A0002CC001F02DC002F001500E24196E025034
:1004B0000F201A6E000E10201B6E000E11201C6EF5
:1004C0001BC044F01CC045F019C05CF01AC05DF0C0
:1004D0008982C5D13E0E175C2EE12184D6CF0EF065
:1004E000D7CF0FF03C0E18240C6E0D6A0D36185045
:1004F0000C24016E000E0D20026E01C02EF002C011
:100500002FF02EC001F02FC002F001500E24196E02
:1005100002500F201A6E000E10201B6E000E1120CC
:100520001C6E1BC046F01CC047F019C05EF01AC01C
:100530005FF0898094D13F0E175C2EE12186D6CFE3
:100540000EF0D7CF0FF03C0E18240C6E0D6A0D364E
:1005500018500C24016E000E0D20026E01C030F008
:1005600002C031F030C001F031C002F001500E2461
:10057000196E02500F201A6E000E10201B6E000E16
:1005800011201C6E1BC048F01CC049F019C060F05F
:100590001AC061F0898663D1400E175C2EE1218874
:1005A000D6CF0EF0D7CF0FF03C0E18240C6E0D6A8C
:1005B0000D3618500C24016E000E0D20026E01C085
:1005C00032F002C033F032C001F033C002F001500B
:1005D0000E24196E02500F201A6E000E10201B6E92
:1005E000000E11201C6E1BC04AF01CC04BF019C03D
:1005F00062F01AC063F0898832D1410E175C2EE197
:10060000218AD6CF0EF0D7CF0FF03C0E18240C6EF7
:100610000D6A0D3618500C24016E000E0D20026E6E
:1006200001C034F002C035F034C001F035C002F032
:1006300001500E24196E02500F201A6E000E102069
:100640001B6E000E11201C6E1BC04CF01CC04DF028
:1006500019C064F01AC065F0898A01D1480E175C90
:1006600028E12280D6CF0EF0D7CF0FF0140E182439
:10067000016E026A023601C036F002C037F036C0A1
:1006800001F037C002F001500E24196E02500F2005
:100690001A6E000E10201B6E000E11201C6E1BC067
:1006A0004EF01CC04FF019C066F01AC067F08A8681
:1006B000D6D0490E175C28E12282D6CF0EF0D7CFD4
:1006C0000FF0140E1824016E026A023601C038F0D1
:1006D00002C039F038C001F039C002F001500E24D8
:1006E000196E02500F201A6E000E10201B6E000EA5
:1006F00011201C6E1BC050F01CC051F019C068F0D6
:100700001AC069F08A84ABD04A0E175C28E12284B3
:10071000D6CF0EF0D7CF0FF0140E1824016E026A58
:10072000023601C03AF002C03BF03AC001F03BC0D3
:1007300002F001500E24196E02500F201A6E000EA6
:1007400010201B6E000E11201C6E1BC052F01CC02E
:1007500053F019C06AF01AC06BF08A8280D04B0E39
:10076000175C28E12286D6CF0EF0D7CF0FF0140EFB
:100770001824016E026A023601C03CF002C03DF04E
:100780003CC001F03DC002F001500E24196E025031
:100790000F201A6E000E10201B6E000E11201C6E12
:1007A0001BC054F01CC055F019C06CF01AC06DF09D
:1007B0008A8055D04C0E175C28E12288D6CF0EF0E7
:1007C000D7CF0FF0140E1824016E026A023601C052
:1007D0003EF002C03FF03EC001F03FC002F00150C9
:1007E0000E24196E02500F201A6E000E10201B6E80
:1007F000000E11201C6E1BC056F01CC057F019C013
:100800006EF01AC06FF08B8A2AD04D0E175C27E16C
:10081000228AD6CF0EF0D7CF0FF0140E1824016E17
:10082000026A023601C040F002C041F040C001F04F
:1008300041C002F001500E24196E02500F201A6EB2
:10084000000E10201B6E000E11201C6E1BC058F0F5
:100850001CC059F019C070F01AC071F08B8817686D
:100860002152D8B4AED021A01BD042C01BF043C04F
:100870001CF05AC019F05BC01AF0D6CF0EF0D7CFDB
:100880000FF019500E5C1A500F581B5010581C5086
:10089000115811501C18D8B0800A02E78994219091
:1008A00021A21BD044C01BF045C01CF05CC019F055
:1008B0005DC01AF0D6CF0EF0D7CF0FF019500E5CF6
:1008C0001A500F581B5010581C50115811501C181A
:1008D000D8B0800A02E78992219221A41BD046C099
:1008E0001BF047C01CF05EC019F05FC01AF0D6CFF5
:1008F0000EF0D7CF0FF019500E5C1A500F581B5046
:1009000010581C50115811501C18D8B0800A02E71A
:100910008990219421A61BD048C01BF049C01CF02F
:1009200060C019F061C01AF0D6CF0EF0D7CF0FF02B
:1009300019500E5C1A500F581B5010581C5011586B
:1009400011501C18D8B0800A02E78996219621A878
:100950001BD04AC01BF04BC01CF062C019F063C032
:100960001AF0D6CF0EF0D7CF0FF019500E5C1A50F8
:100970000F581B5010581C50115811501C18D8B04B
:10098000800A02E78998219821AA1BD04CC01BF04D
:100990004DC01CF064C019F065C01AF0D6CF0EF03F
:1009A000D7CF0FF019500E5C1A500F581B5010582B
:1009B0001C50115811501C18D8B0800A02E7899AAF
:1009C000219A2252D8B4AED022A01BD04EC01BF028
:1009D0004FC01CF066C019F067C01AF0D6CF0EF0F9
:1009E000D7CF0FF019500E5C1A500F581B501058EB
:1009F0001C50115811501C18D8B0800A02E78A9672
:100A0000229022A21BD050C01BF051C01CF068C025
:100A100019F069C01AF0D6CF0EF0D7CF0FF01950E9
:100A20000E5C1A500F581B5010581C501158115082
:100A30001C18D8B0800A02E78A94229222A41BD004
:100A400052C01BF053C01CF06AC019F06BC01AF002
:100A5000D6CF0EF0D7CF0FF019500E5C1A500F58AA
:100A60001B5010581C50115811501C18D8B0800A37
:100A700002E78A92229422A61BD054C01BF055C0D4
:100A80001CF06CC019F06DC01AF0D6CF0EF0D7CFA5
:100A90000FF019500E5C1A500F581B5010581C5074
:100AA000115811501C18D8B0800A02E78A9022967B
:100AB00022A81BD056C01BF057C01CF06EC019F006
:100AC0006FC01AF0D6CF0EF0D7CF0FF019500E5CD2
:100AD0001A500F581B5010581C50115811501C1808
:100AE000D8B0800A02E78B9A229822AA1BD058C05D
:100AF0001BF059C01CF070C019F071C01AF0D6CFAD
:100B00000EF0D7CF0FF019500E5C1A500F581B5033
:100B100010581C50115811501C18D8B0800A02E708
:0A0B20008B98229A2DEF01F0FFD709
:020000040030CA
:0300010006170ED1
:020005008580F4
:060008000FC00FE00F40E5
:00000001FF
